:030000000219FDE5
:03000B000200AA46
:03002B0002019936
:03005B0002034C51
:0300730002033253
:1000800002030406080C10182030406080040608A3
:100090000C10182030406080A0C000070F1F3F0DDB
:1000A0000D04050D050305030302C2AF306308C24A
:1000B00063857C8AD2AF32C0D0C0E0206227E525BC
:1000C0006002E473E525F4C3334009758A00D26306
:1000D000F57C01D6F58A758B00758D00D262D0E073
:1000E000D0D0D2AF32C3E526334009758A00D2633F
:1000F000F57C01F6F58AC262E526F4603B306803C0
:10010000207213758B00758D00D0E0D0D0C292C2E2
:1001100094C296D2AF32C292C294C296206E0C2084
:100120006609740AD5E0FDE57E4290758B00758DF9
:1001300000D0E0D0D0D2AF32758A00D263757C0097
:10014000C28DD262212B01C4306805206602D29292
:1001500001C4306805206602D29401C430680520CD
:100160006602D29601C4C29330680A2066077408FA
:10017000D5E0FDD29201C4C29530680A20660774AA
:1001800008D5E0FDD29401C4C29730680A20660702
:100190007408D5E0FDD29601C4C2AFC2AD53E6EFFC
:1001A000C0D0C0E0D2D3D2AFE57D6009E57A60056A
:1001B000757A0041DF757A01C2CEE52A60072074A6
:1001C00049152A410A7800790020742EE580307E96
:1001D00001F430E60278FF53DACF207E0343DA20C1
:1001E000307E0343DA10C2D8C271E580307E01F45C
:1001F00030E60279FFC3E89970CB306103752A18A5
:10020000207403752A18885FD27020740DE52B6066
:1002100004152B411A43DA01C2D82070024178A894
:100220005F206102C2702074367982B70431C3E85E
:1002300094F0400374F0F8E8C4540F28F87984B7B8
:100240000302415FC313C3138721200802C3132095
:100250000A06C3C898F8415F28F8500374FFF8886D
:1002600022E52D54066011E533C313C3132406257C
:1002700022F52250037522FF7882B6045985222484
:10028000A824C3E52495644002A864C3E8956640A9
:1002900002A8668825E569700241C9C3E8AA699A7F
:1002A0005003E8FAE4F9EAC333FBE56BF45B294059
:1002B0000D256AF8E56A6002156A400B41C90AC358
:1002C000E56A9A5002056A78FF8826C26EC3E52661
:1002D00094F84002D26EC3E52594404002D26420D7
:1002E000CF0AD0E0D0D043E610D2AD32C2CF053A2B
:1002F000E57D6009E57B6005757B006128757B0104
:100300007801E52A6005307402152AC3E55F94017F
:1003100040057562006128756300756C00E5622414
:1003200001F56250037562FFD0E0D0D043E610D2F1
:10033000AD32C2AFC0D053E67FC260759100855622
:1003400094855795759104D0D0D2AF32C2AF53E6A1
:10035000EFC2ADC0D0C0E0C0F0D2D3D2AFA8FBA9ED
:10036000FCE57D6007C3E913F9E813F8C2D83071E2
:100370000261BE53DACF207E0343DA10307E03439E
:10038000DA20D271E580307E01F420E602619588A2
:10039000278928A1E553DACF207E0343DA20307E77
:1003A0000343DA10C2D8C271307402A1D17800E5DB
:1003B00080307E01F430E602A1D1885FA1B953DA22
:1003C000CF207E0343DA20307E0343DA10C271204F
:1003D0006102819753DACF207E0343DA10307E0327
:1003E00043DA20C2D8D271885A895BC3E89558F89D
:1003F000E99559F97B007E087A00C3E8948CE9946A
:10040000005005755E008189882178A2E6A82160E8
:1004100055C3E894C8E994005008E4D2E4FB7A0A92
:100420008164C3E89468E994015008E4D2E3FB7A5C
:100430000F8164C3E894D0E994025008E4D2E2FB4F
:100440007A1E8164C3E894A0E994055008E4D2E1DF
:10045000FB7A3C8164C3E89498E994085008E4D29C
:10046000E0FB7A787E00C3E8955CFCE9955DFD30A1
:0F047000E70AECF42401FCEDF43400FD755E00A6
:10047F00C3EC9AED9E5003755E01885C895D855AC9
:10048F0058855B597802A1B9C3E89527F8E99528F3
:10049F00F9307C02A19D307B02A19D307A02A1969A
:1004AF0020750281BAE9FDE8FC81D9E9C313F9E8A7
:1004BF0013F8307902A196E9C313F9E813F83078ED
:1004CF0002A196E9C313FDE813FC206126C3EC9447
:1004DF001CED9402400281F0ED7018C3EC94C850EB
:1004EF00120529C3E529940A5002A1D1755F00D2E4
:1004FF0070A1D1E529600215297888E6F9740020EA
:10050F007F087896B90302789EE624FAFEE4340059
:10051F00FFC3EC9EFCED9FFD9208B90310A208509B
:10052F0007207609D276A13C307602C276A2085017
:10053F0016B9030DECF42401FCEDF43400FD0205B3
:10054F005678007900A19DB90315EC33FCED33FD0E
:10055F00C3EC940AFCED9400FD50047C007D00C3B5
:10056F00EC94FFED9400400678FF7900A19DEC8597
:10057F0075F0A4C5F0A2F733F8790040030205B96E
:10058F0078FF79000205B9E9C313F9E813F8307C55
:10059F000EE9600278FFC3E81338F8E43400F9C3BA
:1005AF00E894FFE99400400278FF885FD2702061E1
:1005BF0002A1D1741FF4552F4BF52FC274EB7002AB
:1005CF00D274752A18307403752A0A306102A1E5B6
:1005DF0020740353DAFE207403752B06D0F0D0E09D
:1005EF00D0D0D2AD43E6103279010206157903025D
:1005FF000615790A020615791E0206157964020698
:10060F001579C80206157817E4D5E0FDD8FAD9F6A2
:10061F00227A147B7802063C7A107B8C02063C7A95
:10062F000D7BB402063C7A0B7BC802063C7902B202
:10063F007DE4C295D5E0FDD294D5E0FDC294D5E01E
:10064F00FDD295D5E0FDD292E576D5E0FDC292744C
:10065F0096D5E0FDD9D9EAF8D5E0FDD8FBDBCEC2BF
:10066F009522C37C007D0075F00005F0EA33FAEBAC
:10067F0033FB50F6EB13FBEA13FAC3E9FFE8FEE88E
:10068F009AF8E99BF95004EFF9EEF8B3EC33FCED6F
:10069F0033FDD5F0DFEDF9ECF822E889F08A20D2AE
:1006AF00D4F8A9F07B0030F70B7BFFF42401F8E9B5
:1006BF00F43400F9E88520F0A4ADF0F8E98520F0D6
:1006CF00A4AFF0FEED2EF974003FFA7C04C3EA13D9
:1006DF00FAE913F9E813F8DCF48BF030F70AE8F4D1
:1006EF002401F8E9F43400F9E889F0C2D4F8A9F04C
:1006FF00227882B6040302075BC3E55F94014003CF
:10070F00020725852224E4F545F546F547F548F51A
:10071F0049C26D02075B7882E6FCD26DE522F523B4
:10072F00783879C7AA40AB41C3EB13FBEA13FAEC55
:10073F00146013C3EB13FBEA13FAEC14146007C332
:10074F00EB13FBEA13FAD1718845894622C3E545BD
:10075F009523F8E5469400F9500CC3E89480E9948A
:10076F00FF401602078CC3E8947FE9940050030200
:10077F00078C787F790002078C788079FF884A8907
:10078F004B22E54A2547F8E54B3548F9854B20E4E0
:10079F00300701F43549FA30E709C3EA94F0401500
:1007AF000207CAC3EA940F50030207CA78FF79FF02
:1007BF007A0F0207CA780079007AF0C3E5249564AE
:1007CF00500AC374019524500B0207E8E54B20E74C
:1007DF000E0207E8E54B30E706884789488A492229
:1007EF0078A4E6FAC3E54A33F8E54B33F9D1A9E922
:1007FF0030E70BC3E89480E994FF40130122C3E86C
:10080F00947FE9940050020122787F7900012278C9
:10081F008079FFE820E715C3E52398F84009C3E87E
:10082F00940140030208497801020849E8F42401C1
:10083F002523F8400302084978FF884C2278A5E663
:10084F00FAA848A9491206A9E930E70CC3E89401B0
:10085F00E994FF401602087EC3E894FFE994005024
:0F086F000302087E78FF790002087E780179FF86
:10087E00E920E715C3E54C98F84009C3E894014018
:10088E00030208A578010208A5E8F42401254CF816
:10089E0040030208A578FF88242278FFC2642069ED
:1008AE003D206A12D264C3E541940A4009C3E5258E
:1008BE0094405002C26479A1E76023E541601F7441
:1008CE00FF8541F0848539F0306A0375F005A4F890
:1008DE00C5F0600278FFC3E895675002A867886686
:1008EE0022C3E54094C8E5419400E5665003142107
:1008FE0000046002F566220209082275E89022784B
:10090E0083E6FFE5E820ECF7A8BDA9BE0573C3E5B5
:10091E007394084052757300E9FA79A0E76044EACF
:10092E007007E574601B020943C3E895746010E517
:10093E00745006600C1402094F0460F902094FE569
:10094E0074F574C39472401B7564C0C39404401351
:10095E00756480C39404400B756440C394044003D3
:10096E0075640075BB0922E5642410500274FFF50E
:10097E00647982B70402219CC3A864E524985002CE
:10098E00A824C3E895664002A86688258826E573E4
:10099E00B4070375BB1022743279A687F0A4C5F094
:1009AE00A2F733F8C3E895644002A864882288242D
:1009BE00882588268867227540007541F022C2AFCF
:1009CE0075C820A8CCA9CDAA3A30CF010A75C82483
:1009DE00D2AFC3EA13FAE913F9E813F8AB3BAC3C18
:1009EE00883B893CC3E89BF8E99C20690A547FF94F
:1009FE0030670241EF414CAD3D8A3DF9EA9D547F8F
:100A0E00FA600478FF79FFAE3EAF3F8B3E8C3FC35A
:100A1E00EC9FFCC3E99CF542A83BA93CC3E89EF8B9
:100A2E00E99FF9C3E54113FBE54013FAE82AF540C7
:100A3E00E93BF54150067540FF7541FF4196AA40CE
:100A4E00AB41AC40AD417E047F02C3EB9404400247
:100A5E001E1FC3EB940840021E1FC3ED13FDEC13C3
:100A6E00FCDEF7C3EA9CFAEB9DFBEF6009C3E913CA
:100A7E00F9E813F8DFF7EA28FAEB39FB8A408B41E5
:100A8E0050067BFF8B408B41C3EB94025002D26722
:100A9E003069047F0341C17892E6FFC3E537948243
:100AAE0040110FC3E53794A040010FC3EF940640E9
:100ABE00027F057E02E541C4540FF9E541C454F0AE
:100ACE00F8E540C4540F28F8C3E89EFAE99400FBF9
:100ADE004009C3EA9402EB940050047A02E4FB61ED
:100AEE003BAA40AB41EBC4FEEAC4540F4EFCC3EA32
:100AFE009CFAEB9400FBC3E813C313F8EA28FAEB55
:100B0E003400FB8A408B41C3EB94024002C26778EB
:100B1E0002EBC4FE7B00EAC4540F4EFAC3EA98FA05
:100B2E004005C3940250027A027892E6FF306002CA
:100B3E00613B855256855357D26043E680C3E49A93
:100B4E00F8E49BF9C3E833F8E933F930670261DC66
:100B5E00E8FAE9FBD3E913FDE813FC88528953C385
:100B6E00EF94036038EF20E00DE82CF8E93DF9EC46
:100B7E00FAEDFB020B97E828F8E939F9C3E82402ED
:100B8E00F8E93400F97AFE7BFFC3EF9403400E8A36
:100B9E00548B55884E894F8C508D518110885489B5
:100BAE00558A4E8B4F8C508D51306920C3E533944E
:100BBE00034019E542A2E713F8E555F42401384045
:100BCE000B20E7087554FFF42401F5558110E8FA5F
:100BDE00D3E813FC8852C3EF94036020EF20E007A4
:100BEE00E82CF8ECFA61FCE8282402F87AFEC3EF50
:100BFE00940340088A54884E8C50811088548A4E33
:100C0E008C50E56BC3335002646BF56B3060028120
:100C1E001A753404D26043E680E52D5406601FA891
:100C2E0040A941C2AF53E67F759100C3E498F59495
:100C3E00E499F595759104D26043E680D2AF22D245
:100C4E0065754400752000306B03752040020C6CF6
:100C5E00D265754400752040306B03752000D2AF0D
:0E0C6E007801206722E52D54066002C265C39E
:100C7C00E5419405401378029405400878039405E7
:100C8C0040027806306902780A206019E544601544
:100C9C0030690AC3E53394034003D53406D2AFD28E
:100CAC006CA14E9122D2AF0000C2AF20672AE54161
:100CBC00C3FB940F40027B0FEB24053073012330F0
:100CCC006A02742820620123F93069027982E58D69
:100CDC0013E58B13C39940B10544E59B5440B520F3
:100CEC0002A13830690A08C3E8940A4001088195CA
:100CFC00206502816CC26553E67F759100306710E8
:100D0C007594007595FC759104D26043E680816CF6
:100D1C00AE40AF41C3EE33FEEF33FF50047EFF7F96
:100D2C00FFC3E49EF594E49FF595A112C3E53394BB
:100D3C00025002816C306502816CD802A14C819505
:100D4C00C26C53E67F7591008554948555957591C9
:100D5C0004854E56854F57D26043E680D2AFE52DC1
:100D6C0054066008206A020533020D88306C0D2091
:100D7C006B0A206507158115810216282278003030
:100D8C0064053065027801E53775F007A4F9E5F0E4
:100D9C0028F5F0E9A2F013A2F113A2F213F537C370
:100DAC0094785003753778C3E53795384008D26688
:100DBC00C292C294C296306002A1C285505685512F
:100DCC0057D26043E68022D287207D11C2AF754393
:100DDC0002C295D293D2AF759F80020FAEC2AF758F
:100DEC004302C295D297D2AF759F80020FAEC287D5
:100DFC00307243207D20C2AF754303900177757E1E
:100E0C0020C296C297306204D294C11AD295D2AF46
:100E1C00759F89020FAEC2AF754303900177757E43
:100E2C0020C292C293306204D294C13AD295D2AF0E
:100E3C00759F81020FAE207D17C2AF7543039001E1
:100E4C0052C296306202D294D2AF759F89020FAE15
:100E5C00C2AF754303900152C292306202D294D257
:100E6C00AF759F81020FAED287207D11C2AF754343
:100E7C0004C293D297D2AF759F81020FAEC2AF75E9
:100E8C004304C297D293D2AF759F89020FAEC2872B
:100E9C00307243207D20C2AF754305900166757E8C
:100EAC0008C294C295306204D292C1BAD293D2AF26
:100EBC00759F80020FAEC2AF754305900188757E99
:100ECC0080C294C295306204D296C1DAD297D2AF66
:100EDC00759F80020FAE207D17C2AF754305900140
:100EEC0048C294306202D292D2AF759F80020FAE8C
:100EFC00C2AF75430590015CC2943062EBD296D2BE
:100F0C00AF759F80020FAED287207D11C2AF7543A3
:100F1C0006C297D295D2AF759F89020FAEC2AF753C
:100F2C004306C293D295D2AF759F81020FAEC28792
:100F3C00307242207D20C2AF754301900188757ECE
:100F4C0080C292C293306204D296E15AD297D2AF49
:100F5C00759F81020FAEC2AF754301900166757E1D
:100F6C0008C296C297306204D292E17AD293D2AF81
:100F7C00759F89E1AE207D16C2AF75430190015C6F
:100F8C00C292306202D296D2AF759F81E1AEC2AFEF
:100F9C00754301900148C296306202D292D2AF756D
:100FAC009F89C26622900146757E00C292C294C28D
:100FBC0096C293C295C297C262227880760908764F
:100FCC00090876040876FF0876030876FF08760988
:100FDC00087603087601087601788C76010876FF8E
:100FEC000876FF0876FF0876FF0876FF0876030878
:100FFC0076FF0876FF0876FF0876250876D0087607
:10100C00280876500876040876FF087602087600E1
:10101C0008767A0876FF08760108760108760008CB
:10102C007603227887E6FFC272BF0302D2727888F9
:10103C00E6C394036008C27DE630E102D27DC27E35
:10104C007889E630E102D27EC3EF94026008758E97
:10105C0001D273021067758E00C273227880E61479
:0F106C009000809378A4F67881E614900080932A
:10107B0078A5F67886E61490008D9378A6F6789C82
:10108B00E67538FF75390CB402067538A075390A48
:10109B00B4030675388275390578A3E61490009A67
:1010AB0093F569120FB122C2A4C2A0789DE6B401D8
:1010BB0004D2A4C2A0B40204C2A4D2A0227896E6A1
:1010CB00FA7897E6FB7888E6B40305C3EB940EFB3E
:1010DB00307F047A007BFFC3EB9AFCC394825002EF
:1010EB007C827575000575EC8575F0A4C3E5F094ED
:1010FB007D40F222D27F11C81206067A007B007C5B
:10110B00101205FCE55F2AFA74003BFBDCF37C0450
:10111B00C3EB13FBEA13FADCF7FEC27F11C822E51F
:10112B00EF20E6037520000520903FFFE5201460BB
:10113B0006901FFF1460009304600375EF1253D9E0
:10114B00BF7581C043FF801205F775EF0243B203F1
:10115B00E5B3240420E70DF521E5E320E006852126
:10116B00B343E301120FB17580FF75A48075F1F0E5
:10117B0075D4BF75900275A5FC75F2FD75D502751A
:10118B00A61175A0EE75F3F175E241E4F8F6D8FD02
:10119B00756B01120FC61216727898867675300130
:1011AB00C2AF1206101206201206061206271206EE
:1011BB000612062E120606C2AF78FA79FA308607A7
:1011CB00D9FBD8F7021C00112F116811B211C87886
:1011DB00988676120FB175B68075A900757D00756E
:1011EB00885075891275C82475910475D84075A8F7
:1011FB002275B80275E690759B80759D0075D10EB2
:10120B0075BC5875BB0975BA1175E8801205F7D214
:10121B00AF12090553DACF207E0343DA20307E0369
:10122B0043DA1043DA01C2D8C271120610D2617BC5
:10123B00037A0CE55E70077A0CDB030211C212060F
:10124B00062070030211C2C270E55FC3940240E135
:10125B00E52F541F856160F561B560D5DAD5C261A4
:10126B0053DACF207E0343DA20307E0343DA10C2F9
:10127B00D8C27178A2E67008D274E52F54E0F52F2E
:10128B00C27575290012060B307409C3E529940A3F
:10129B004002D2751205FC78023074027800C3E567
:1012AB005F9840F0C2AF120620120620120620D221
:1012BB00AF120610754D007888E6B4030261A012D8
:1012CB0005FC788CE6C3940150030213A0E530C3F0
:1012DB00940150030213A0207435C3E55F94FF50B3
:1012EB00030213A0C2AF120635D2AF12060BC3E531
:1012FB005F940150EFC2AF120620120601120620B6
:10130B00D2AF12060BC3E55F94FF40E902181A7FB8
:10131B0002D27F11C812060BC2AFC27F11C8AE5FDB
:10132B00C3E55F947FD2AF40761205F7C2AF1206CA
:10133B0035D2AFDFDC11FFC3EE94057897F61206BA
:10134B00101216B412179D7F0AD27F11C812060B0A
:10135B00C2AFC27F11C8AE5FC3E55F947FD2AF50FF
:10136B00E61205F7C2AF120620120601120620D2B2
:10137B00AFDFD611FFEE24057896F6120610121683
:10138B00B41217CC12060B11C8C3E55F94FF5002C1
:10139B0041E202181AC3E55F954D4003855F4D127C
:1013AB00060B78017988E7B403027805C3E55F98EB
:1013BB00400241C2C2AF120635120635120635D2B3
:1013CB00AF120610753000E4F531F5320531E53119
:1013DB00F470390532789AE6781914601278321461
:1013EB00600D787D14600878FA146003753200C3C1
:1013FB00E53298401715327531B478998676C2AFBD
:10140B00120635D2AF7898867612060B120601E5D6
:10141B002A700530740221C278012074027806C349
:10142B00E55F9840A77888E6C39403600312060B28
:10143B00E52A70030211C2C2AF120FB1E4F522F517
:10144B0023F524F525F526F56AD2AF7885E6C33367
:10145B00F568E4F545F546F547F548F549F573F5B7
:0E146B002CF52DF53775730875BB101205F7BB
:10147900120909E5E820ECFBA8BDA9BEE97001F84D
:10148900887412090D75730875BB107887E6FE76A6
:1014990002112F7887EEF6C2AF7564FF1209A58590
:1014A9002264852265852266D2AF752201752401E1
:1014B90075250175260185636C756D0175B6907585
:1014C900A903757D017888E6B40307C27D307602E9
:1014D900D27DD268D269753300120F13120F3A12F6
:1014E90009C51209CC1209C51209CC1209C5021580
:1014F90006C2AF112FD2AF75730075BB09120C5E0E
:10150900120700120D89120DD31209CC120C4D309D
:101519006D0312075C2067031208A83067031208DD
:10152900EF120D89120DFA1209CC120C5E306D03FF
:10153900120791120D89120E731209CC120C4D303B
:101549006D031207EF120D89120E9A1209CC120CB3
:101559005E306D0312084C120D89120F131209CC5B
:10156900120909120C4D120D89120F3A12090D12A6
:1015790009CC306935206B32856764856765856379
:101589006C756D0179187A0CC3E53399400FC269FE
:10159900D26A8A358567648567660215B3C3E55FD4
:1015A90094014003021506021630306A1B206B189D
:1015B900E535147004C26A81FAF535C3E55F940113
:1015C9004003021506021630753600C3E56278FA43
:1015D900985054307404E52A604D7888E6B40317AE
:1015E900207D05207607C100307602C100206B07F7
:1015F900D26B856764A14578F0306B05856764789F
:1016090020C3E541985002A106306B1BC26BC27D15
:10161900307602D27DD26A753512856764A10605D6
:1016290036E55F6002C133753600C2AF120FB1787B
:1016390087E6FE7602112F7887EEF6E4F522F52388
:10164900F524F525F526F568C26875B68075A900F3
:10165900757D00D2AF1205F7120FB1307409C3E5D9
:10166900369405400221C261D2901A0D78201216D3
:10167900F6E520B4550CA31216F6E520B4AA030228
:101689001694120FC61216B40216B3901A03788074
:101699007B0A1216F6A308DBF9901A0F788C7B18CF
:1016A9001216F6A308DBF9901A2722C2AF121735D2
:1016B90012170F901A00740E1216FBA37404121657
:1016C900FBA374141216FB901A0378807B0A121676
:1016D900FAA308DBF9901A0F788C7B181216FAA373
:1016E90008DBF9121748121726901A2722E493F6F5
:1016F90022E6438F01538FFD75EF0275B7A575B7C4
:10170900F1F0538FFE22438F02438F0175EF02756B
:10171900B7A575B7F1901A0DF0538FFC22901A0DE9
:101729007455D1FB901A0E74AAD1FB227A3079D064
:101739007820901A40D1F6E520F709A3DAF7227A42
:101749003079D0901A40E7D1FB09A3DAF922AB77B7
:10175900A878BB01027980BB02027981BB030279B7
:1017690082BB04027984BB05027986BB06027992A1
:10177900BB07027987BB080279A3BB0902799CBB25
:101789000A027988BB0B027989E8F7227C051206DF
:1017990010DCFB22C2AF12062012062712062E12F7
:1017A900063512060112062012062712062E120607
:1017B9003512060112062012062712062E120635C8
:1017C900D2AF22C2AF12063512062E120627120612
:1017D9002012060112063512062E120627120620BD
:1017E90012060112063512062E120627120620D2FB
:1017F900AF22AE77AF78C2AF1206201206201206CA
:1018090020120601DEF2120635120601DFF8D2AF08
:101819002212179D12179512179575770175780180
:101829007579001217FB7C05AD5F120610C3ED95A3
:101839005F70F5C3E55F9401400AC3E55F94FF401B
:101849003702185E1217571216B412179DC2AF75D8
:10185900EF12121795DCD10579C3E579940350028B
:0F18690080C11217950578E5771490009F93F8CA
:1018780008C3E57898500280A812179512179505A5
:1018880077C3E577940C50028094120FC61216B4F1
:08189800C2AF75EF12121795A3
:0319FD0002112AAA
:101A00000E0414090904FF03FF0903010155AA018B
:101A1000FFFFFFFFFF03FFFFFF25D0285004FF0259
:081A2000007AFF01010003FF41
:101A400023506C6174696E756D3530417633232097
:101A500023424C48454C492346333930232020202B
:101A60002020202020202020202020202020202076
:101C0000C2AFC2D353D9BF7581C043B20343FF8073
:101C1000752438752503B1C975EF0275E24043F1AB
:101C20004053A4BF75D400D2867DFA780379E67C50
:101C300010752200752300901DD67B0675249875BB
:101C400025013086028142208608D8FBD9F9DCF7CD
:101C500081B4308608D8FBD9F9DCF781B4B189E4C6
:101C600093A3C39A6004DDC381B4DBDBB17B600264
:101C7000812B7B08E493FAA3B15CDBF87A30B15C8A
:101C8000752200752300B17BEAFCEBFDC3ED94FEE9
:101C9000400EB17B8A278B28ED30E0048A828B834B
:101CA000B17B7AC270D8C3ED94FE601350CEBD00F4
:101CB00025EC60097520007521FF0200008100A855
:101CC00027A9280809D804D90281D3B17FEA89AAB3
:101CD000F281C50D81A0C3ED94035049EDA2E092BD
:101CE000007AC5C3E5829400E583941C50902000DF
:101CF00010438F02438F0175B7A575B7F1F030001F
:101D00001FA827A9280809438F01538FFDD804D99C
:101D100002A12089AAE275B7A575B7F1F0A3A10DBC
:101D2000538FFC817C7AC1BD030CE493A3FAB140CC
:101D3000DCF8B138817C817EAA22AB23B15CEBFA5E
:101D4000EA6222752608C3E52313F523E52213F57D
:101D50002250066323A0632201D526EAB1C9B1C986
:101D600075260AEAF4200102D286300102C286B149
:101D7000C9C3134002C201D526EB22B17FEAFB2082
:101D80008602A17F308602A184752608AE24AF2585
:101D9000C3EF13FFEE13FEB1CDB1C9C3EA13308612
:101DA000024480FA30E703632201C3E52313F523DD
:101DB000E52213F52250066323A0632201D526D91C
:101DC000E52265236523F52222AE24AF250E0FDE22
:101DD000FEDFFCD20122424C48656C693437316326
:041DE000F390060175
:00000001FF
